:020000040800F2
:1000000000070020F5040008912F0008492F000880
:10001000712F0008492F0008692F0008F704000815
:10002000F7040008F7040008F7040008853F0008FB
:10003000F7040008F7040008F7040008F7040008B4
:10004000F7040008F7040008F7040008F7040008A4
:10005000F7040008F704000831530008595300085A
:1000600081530008A9530008D1530008F704000881
:10007000F7040008F7040008F7040008F704000874
:10008000F7040008F7040008F7040008D92E000858
:10009000E92E0008FD2E0008F7040008F9530008B7
:1000A000F7040008F7040008F7040008F704000844
:1000B000E1540008F7040008F7040008F7040008FA
:1000C000F7040008F7040008F7040008F704000824
:1000D000F7040008F7040008CD540008F7040008EE
:1000E0005D540008F7040008F7040008F70400084E
:1000F000F7040008F7040008F7040008F7040008F4
:10010000F7040008F7040008F7040008F7040008E3
:10011000F7040008F7040008F7040008F7040008D3
:10012000F7040008F7040008F7040008F7040008C3
:10013000F7040008F7040008F7040008112F00086E
:10014000212F0008352F0008F7040008F7040008E5
:10015000F7040008F7040008F7040008F704000893
:10016000F7040008F7040008F7040008F704000883
:10017000F7040008F7040008F7040008F704000873
:10018000F7040008F7040008F7040008F704000863
:10019000F7040008F7040008F7040008F704000853
:1001A000F7040008F7040008F7040008F704000843
:1001B000F7040008F7040008F7040008F704000833
:1001C000F7040008F7040008F7040008F704000823
:1001D000F7040008F7040008F7040008F704000813
:1001E000A51800080000000000000000000000004A
:1001F00053B94AB9002908BF00281CBF4FF0FF318E
:100200004FF0FF3000F074B9ADF1080C6DE904CE89
:1002100000F006F8DDF804E0DDE9022304B07047E1
:100220002DE9F047089D04468E46002B4DD18A42A9
:10023000944669D9B2FA82F252B101FA02F3C2F1DC
:10024000200120FA01F10CFA02FC41EA030E94406D
:100250004FEA1C48210CBEFBF8F61FFA8CF708FB8E
:1002600016E341EA034306FB07F199420AD91CEB66
:10027000030306F1FF3080F01F81994240F21C8198
:10028000023E63445B1AA4B2B3FBF8F008FB1033E0
:1002900044EA034400FB07F7A7420AD91CEB040415
:1002A00000F1FF3380F00A81A74240F207816444E5
:1002B000023840EA0640E41B00261DB1D44000236A
:1002C000C5E900433146BDE8F0878B4209D9002DCE
:1002D00000F0EF800026C5E9000130463146BDE858
:1002E000F087B3FA83F6002E4AD18B4202D38242C2
:1002F00000F2F980841A61EB030301209E46002D71
:10030000E0D0C5E9004EDDE702B9FFDEB2FA82F2C5
:10031000002A40F09280A1EB0C014FEA1C471FFA23
:100320008CFE0126200CB1FBF7F307FB131140EA0A
:1003300001410EFB03F0884208D91CEB010103F1D7
:10034000FF3802D2884200F2CB804346091AA4B299
:10035000B1FBF7F007FB101144EA01440EFB00FE6D
:10036000A64508D91CEB040400F1FF3102D2A645D2
:1003700000F2BB800846A4EB0E0440EA03409CE771
:10038000C6F12007B34022FA07FC4CEA030C20FA1E
:1003900007F401FA06F31C43F9404FEA1C4900FA3E
:1003A00006F3B1FBF9F8200C1FFA8CFE09FB1811BB
:1003B00040EA014108FB0EF0884202FA06F20BD92E
:1003C0001CEB010108F1FF3A80F08880884240F27E
:1003D0008580A8F102086144091AA4B2B1FBF9F0C2
:1003E00009FB101144EA014100FB0EFE8E4508D9BD
:1003F0001CEB010100F1FF346CD28E456AD9023842
:10040000614440EA0840A0FB0294A1EB0E01A14226
:10041000C846A64656D353D05DB1B3EB080261EB94
:100420000E0101FA07F722FA06F3F1401F43C5E96E
:10043000007100263146BDE8F087C2F12003D840A4
:100440000CFA02FC21FA03F3914001434FEA1C47E6
:100450001FFA8CFEB3FBF7F007FB10360B0C43EAD8
:10046000064300FB0EF69E4204FA02F408D91CEB88
:10047000030300F1FF382FD29E422DD90238634486
:100480009B1B89B2B3FBF7F607FB163341EA034126
:1004900006FB0EF38B4208D91CEB010106F1FF3875
:1004A00016D28B4214D9023E6144C91A46EA00466C
:1004B00038E72E46284605E70646E3E61846F8E6FE
:1004C0004B45A9D2B9EB020864EB0C0E0138A3E747
:1004D0004646EAE7204694E74046D1E7D0467BE728
:1004E000023B614432E7304609E76444023842E7A0
:1004F000704700BF02E000F000F8FEE772B6374830
:1005000080F30888364880F3098836483649086001
:1005100040F20000CCF200004EF63471CEF2000141
:100520000860BFF34F8FBFF36F8F40F20000C0F23F
:10053000F0004EF68851CEF200010860BFF34F8FF5
:10054000BFF36F8F4FF00000E1EE100A4EF63C71E2
:10055000CEF200010860062080F31488BFF36F8F8D
:1005600004F0F0FC04F082FD4FF055301F491B4AA7
:1005700091423CBF41F8040BFAE71D49184A9142E9
:100580003CBF41F8040BFAE71A491B4A1B4B9A423D
:100590003EBF51F8040B42F8040BF8E7002018495D
:1005A000184A91423CBF41F8040BFAE704F0CEFC34
:1005B00004F0AAFD144C154DAC4203DA54F8041BA8
:1005C0008847F9E700F042F8114C124DAC4203DACB
:1005D00054F8041B8847F9E704F0B6BC0007002074
:1005E000002300200000000808ED00E000010020CA
:1005F00000070020805900080023002088230020E5
:1006000088230020C8610020E0010008E401000800
:10061000E4010008E40100082DE9F04F2DED108AF7
:10062000C1F80CD0C3689D46BDEC108ABDE8F08FC0
:10063000002383F311882846A047002004F0F4F833
:10064000FEE704F057F800DFFEE70000F8B501F020
:100650003FF904F011FC074604F060FC0546B8BB06
:10066000204B9F4234D001339F4234D01E4B27F0A1
:10067000FF029A4232D1F8B200F020FF2E4642F239
:10068000107400F021FF08B10024264601F002FD9D
:1006900020B1032000F07CF80024264635B1134B2E
:1006A0009F4203D004F032FC00242646002004F0D0
:1006B000EDFB0EB100F082F801F0A0FA00F070FF3F
:1006C00001F064F9204600F0CDF800F077F8F9E782
:1006D0002E460024D5E704460126D2E7064640F61A
:1006E000C414CEE7010007B0000008B0263A09B0F4
:1006F00008B501F017F9A0F120035842584108BD90
:1007000007B541F21203022101A8ADF8043001F04F
:1007100027F903B05DF804FB38B5302383F3118863
:10072000174803680BB104F03DF9164A144800233A
:100730004FF47A7104F02CF9002383F31188124CE2
:10074000236813B12368013B2360636813B16368B6
:10075000013B63600D4D2B7833B963687BB9022090
:1007600001F0DAF9322363602B78032B07D1636839
:100770002BB9022001F0D0F94FF47A73636038BDD1
:100780008823002019070008A8240020A0230020A7
:10079000084B187003280CD8DFE800F008050208A1
:1007A000022001F0AFB9022001F0A2B9024B0022F1
:1007B0005A607047A0230020A824002010B501F043
:1007C00069FC30B1204B03221A70204B00225A6082
:1007D00010BD1F4B1F4A1C4619680131F8D0043365
:1007E0009342F9D162681C4B9A42F1D91B4B9B682A
:1007F00003F1006303F580339A42E9D204F05AFB17
:1008000004F06CFB002001F0DBF80220FFF7C0FFD2
:10081000134B1A6C00221A64196E1A66196E596C01
:100820005A64596E5A665B6E72B64FF0E0233021FF
:10083000C3F8084DD4E9003281F311889D4683F353
:1008400008881047C4E700BFA0230020A824002088
:100850000000010820000108FFFF0008002300201D
:10086000003802402DE9F04F93B0AC4B00902022AD
:10087000FF210AA89D6801F06BF9A94A1378A3B972
:10088000A848012103601170302383F311880368A5
:100890000BB104F087F8A44AA24800234FF47A7100
:1008A00004F076F8002383F31188009B13B19F4B6B
:1008B000009A1A609E4A009C1378032B1EBF0023E7
:1008C00013709A4A4FF0000A18BF5360D346564639
:1008D000D146012001F016F924B1944B1B68002B7E
:1008E00000F01582002001F01DF80390039B002BFF
:1008F00001DA00F0A7FE039B002BEDDB012001F0E5
:10090000F7F8039B213B162BE3D801A252F823F002
:100910006D09000895090008290A0008D308000895
:10092000D3080008D3080008B30A0008830C0008A5
:100930009D0B0008FF0B0008270C00084D0C000859
:10094000D30800085F0C0008D3080008D10C000889
:100950000D0A0008D3080008150D000879090008E1
:100960000D0A0008D3080008FF0B00080220FFF75B
:10097000BFFE002840F0F581009B0221BAF1000F74
:1009800008BF1C4605A841F21233ADF8143000F040
:10099000E7FF9EE74FF47A7000F0C4FF071EEBDB21
:1009A0000220FFF7A5FE0028E6D0013F052F00F248
:1009B000DA81DFE807F0030A0D10133605230593EB
:1009C000042105A800F0CCFF17E054480421F9E702
:1009D00058480421F6E758480421F3E74FF01C0873
:1009E000404600F0EFFF08F104080590042105A837
:1009F00000F0B6FFB8F12C0FF2D1012000FA07F792
:100A000047EA0B0B5FFA8BFB4FF0000901F0ECF8A3
:100A100026B10BF00B030B2B08BF0024FFF770FE71
:100A200057E746480421CDE7002EA5D00BF00B0375
:100A30000B2BA1D10220FFF75BFE074600289BD0BD
:100A4000012000F0BDFF0220FFF7A2FE00261FFAE2
:100A500086F8404600F0C4FF044690B100214046AD
:100A600000F0D6FF01360028F1D1BA46044641F223
:100A70001213022105A8ADF814303E4600F070FFB5
:100A800027E70120FFF784FE2546244B9B68AB42F5
:100A900007D9284600F096FF013040F06781043501
:100AA000F3E7234B00251D70204BBA465D603E46A0
:100AB000ACE7002E3FF460AF0BF00B030B2B7FF481
:100AC0005BAF0220FFF764FE322000F02BFFB0F195
:100AD0000008FFF651AF18F003077FF44DAF0F4A3F
:100AE000926808EB050393423FF646AFB8F5807F66
:100AF0003FF742AF124B0193B84523DD4FF47A70B4
:100B000000F010FF0390039A002AFFF635AF019B17
:100B1000039A03F8012B0137EDE700BF0023002003
:100B2000A42400208823002019070008A8240020FE
:100B3000A023002004230020082300200C230020F1
:100B4000A4230020C820FFF7D3FD074600283FF468
:100B500013AF1F2D11D8C5F1200242450AAB25F075
:100B6000030028BF424683490192184400F0DEFF8B
:100B7000019A8048FF2100F0EBFF4FEAA8037D496E
:100B80000193C8F38702284600F0EAFF06460028D2
:100B90003FF46DAF019B05EB830537E70220FFF7BC
:100BA000A7FD00283FF4E8AE00F052FF00283FF414
:100BB000E3AE0027B846704B9B68BB4218D91F2F85
:100BC00011D80A9B01330ED027F0030312AA134455
:100BD00053F8203C05934046042205A901F012FA7F
:100BE00004378046E7E7384600F0ECFE0590F2E770
:100BF000CDF81480042105A800F0B2FE06E700231A
:100C0000642104A8049300F0A1FE00287FF4B4AE90
:100C10000220FFF76DFD00283FF4AEAE049800F00F
:100C2000FFFE0590E6E70023642104A8049300F08A
:100C30008DFE00287FF4A0AE0220FFF759FD0028AA
:100C40003FF49AAE049800F0FBFEEAE70220FFF7BB
:100C50004FFD00283FF490AE00F00AFFE1E70220CC
:100C6000FFF746FD00283FF487AE05A9142000F0E9
:100C700005FF04210746049004A800F071FE3946E0
:100C8000B9E7322000F04EFE071EFFF675AEBB0737
:100C90007FF472AE384A926807EB090393423FF63D
:100CA0006BAE0220FFF724FD00283FF465AE27F06D
:100CB00003074F44B9453FF4A9AE484600F082FE11
:100CC0000421059005A800F04BFE09F10409F1E7A5
:100CD0004FF47A70FFF70CFD00283FF44DAE00F0A2
:100CE000B7FE002844D00A9B01330BD008220AA982
:100CF000002000F035FF00283AD02022FF210AA86A
:100D000000F026FFFFF7FCFC1C4803F093FD13B036
:100D1000BDE8F08F002E3FF42FAE0BF00B030B2B32
:100D20007FF42AAE0023642105A8059300F00EFE8F
:100D3000074600287FF420AE0220FFF7D9FC80464A
:100D400000283FF419AEFFF7DBFC41F2883003F0D6
:100D500071FD059800F05EFF464600F045FF3C46F9
:100D6000B7E5064652E64FF0000905E6BA467EE6CC
:100D700037467CE6A423002000230020A086010043
:100D8000094A136849F2690099B21B0C00FB013350
:100D90001360064B186844F2506182B2000C01FBEC
:100DA0000200186080B2704718230020142300202E
:100DB00010B500211022044600F0CAFE034B03CBFD
:100DC000206061601868A06010BD00BF107AFF1F2E
:100DD0002DE9F041ADF54E7D0DF134086CAC40F2DB
:100DE000751207460D460EA80021C8F8001000F045
:100DF000AFFE4FF4C4720021204600F0A9FE02F0BD
:100E0000CFF8254B4FF47A72B0FBF2F0186093E8FC
:100E10000700022384E807000DF5E9702382FFF73D
:100E2000C7FF40F604331D49238406A804F06AFC7A
:100E3000182384F832310DF2E3266B440DF1300CA7
:100E40001A4603CA624530607160134606F108060F
:100E5000F6D141460122204600F0F6FE002303931E
:100E6000AB7E029305F11903019380B20123CDE912
:100E700004800093E97E06A3D3E90023384602F0FC
:100E800057FC0DF54E7DBDE8F08100BFAFF300804B
:100E90009E6AC421818A46EEB024002014570008BF
:100EA0002DE9F0412C4C237ADAB080460D465BBB2D
:100EB00027A9284600F0D8FF0746002842D19DF810
:100EC0009D60C82E3ED801464FF4A662204600F031
:100ED0003FFE4FF48073C4F8F8314FF40073C4F848
:100EE0000C334FF44073C4F8203432460DF19E01A8
:100EF00004F1090000F01AFE26449DF89C30777238
:100F000023720BB9EB7E23728122002106AC27A845
:100F100000F01EFE0122214627A800F0E1FF002379
:100F20000393AB7E029305F1190380B2019328234A
:100F3000CDE904400093E97E05A3D3E900234046B0
:100F400002F0F6FB5AB0BDE8F08100BFAFF30080BD
:100F500026417272DF25D7B798560020F0B5254E8E
:100F60004FF48A7505FB0065F1B096F8D83085F826
:100F7000DC300024D822214685F8E8403AA800F069
:100F8000E7FD06F1090000F0DBFDD5F8E4308DF84F
:100F9000F000C2B206AF06F109010DF1F100CDE992
:100FA0003A3400F0C3FD394601223AA800F0C4FFEC
:100FB00080B2CDE9047008230127CDE9023706F19C
:100FC000D803019330230093317A0B4807A3D3E968
:100FD000002302F0ADFBA04206DD01F0E1FFC5F801
:100FE000E000384671B0F0BD2046FBE778F6339F4D
:100FF00093CACD8D98560020C83400202DE9F04FBB
:10100000274FDFF8A880274E87B0384602F0BCFB98
:10101000034600283DD00024CDE90344ADF8144038
:10102000027B8DF8142099684068029403AA03C2D9
:101030001B681D4D43F000430293A146A2462B6856
:10104000D3F810B001F0AEFF10EB080241F100033D
:101050002846CDF800A002A9D84704F2344440F64F
:1010600068030028C8BF49F0010905F586559C4270
:1010700005F11005E3D1B9F1000F05D0384602F0B3
:1010800087FB86F800A0C0E73378072B04D801332C
:10109000337007B0BDE8F08F014802F079FBF8E744
:1010A000C8340020CD5B0020F834002040420F00FF
:1010B00070B50D4614461E4602F096FA50B9022E3F
:1010C00010D1012C0ED112A3D3E90023C5E90023CE
:1010D000012007E0282C10D005D8012C09D0052CC0
:1010E0000FD0002070BD302CFBD10BA3D3E900231F
:1010F000ECE70BA3D3E90023E8E70BA3D3E9002334
:10110000E4E70BA3D3E90023E0E700BFAFF30080DF
:10111000401DA12026812A0B78F6339F93CACD8DDE
:101120009E6AC421818A46EE26417272DF25D7B7B6
:10113000F017304A39059E5638B505460E4C002149
:10114000013500F065FCA4F82C55B4F82C0500F02E
:1011500047FC78B1B4F82C0500F052FC014648B9C0
:10116000B4F82C0500F054FCB4F82C350133A4F885
:101170002C35EAE738BD00BF98560020F8B50E4C74
:101180000E4F0226A4F5805343F8487C237E3BB9DA
:1011900065692DB1284600F0FBFF284604F0F2F9FE
:1011A000204600F0F5FFA4F58654012EA4F11004AA
:1011B00000D1F8BD0126E5E710560020DC570008F5
:1011C0002DE9F04F8FB000AF05460C4602F00CFA47
:1011D000002849D1237E022B1BD1E38A012B18D191
:1011E00001F0DEFE0646FFF7CBFD03464FF4C87064
:1011F000DFF8C482B3FBF0F206F5167602FB10337B
:1012000016FA83F3C8F80030E37E33B9A34B00220B
:101210001A703C37BD46BDE8F08F07F12401204627
:1012200000F0E0FD0028F4D107F11400FFF7C0FD45
:1012300097F8264007F11401224607F1270004F031
:10124000EBF90028E2D10F2C08D8944B1C70D8F889
:101250000030A3F51673C8F80030DAE797F82410C9
:10126000284602F0B9F9D4E7E38A282B2BD010D80E
:10127000012B23D0052BCCD1BFF34F8F8849894B4D
:10128000CA6802F4E0621343CB60BFF34F8F00BF24
:10129000FDE7302BBDD1844EE17E327A9142B8D148
:1012A000607E3146002291F8DC50854200F0A58036
:1012B0000132042A01F58A71F5D1AAE721462846B0
:1012C000FFF786FDA5E721462846FFF7E9FDA0E7E1
:1012D000B2F8EC507B6005F103094FEA99094FEA37
:1012E0008902D11DC908A8EBC1039D46EB46002128
:1012F000584600F02DFC04F1EE012A4631445846D0
:1013000000F014FC7B6813B9012000F059FB96F83B
:10131000D20000F065FB044630B9307200F098FB53
:10132000204600F04DFBB1E0D6F8D4203AB996F84B
:10133000D200B6F82C25824201D8FFF7FDFED6F880
:10134000D4202A44944208D296F8D200B6F82C252C
:101350000130824201D8FFF7EFFE70685FFA89F230
:10136000594600F0FDFB08B9C54679E0726896F869
:10137000D2002A447260D6F8D42005EB0209C6F8E0
:10138000D49000F02DFB814509D396F8D220D6F8F1
:10139000D4000132001B86F8D220C6F8D400FF2DFD
:1013A0000FD80024347200F053FB204600F008FBF5
:1013B00000F070FE3D4B188108B9FFF7FFF9C546F4
:1013C00027E7BB6896F8D9000AFB0362FB68D2F8EE
:1013D000E41082F8E83001F58061C2F8E030C2F82C
:1013E000E410FFF7BBFDFFF709FE96F8D9200132A4
:1013F00002F0030286F8D920B6E74FF48A7A0AFB96
:1014000002F505F1EA013144204600F0C1FDF86023
:1014100000287FF4FEAE3544012285F8E82001F073
:10142000BFFDD5F8E020D6ED007ADFED216A801A05
:10143000192838BF192040F6B832904228BF10460C
:10144000B8EE677A07EE900AF8EEE77A67EEA67ACA
:10145000DFED186AE7EE267AFCEEE77AC6ED007A51
:1014600096F8D930BB60BA6873680AFB02F4321987
:1014700092F8E81059B1D2F8E4108B42E8463FF4F4
:1014800027AF002182F8E810C2F8E010C546736863
:10149000064A9B0A01331381BBE600BFC13400201A
:1014A00000ED00E00400FA0598560020B02400206A
:1014B000CDCCCC3D6666663FC4340020014B18702D
:1014C000704700BFBC24002030B54FF000542B4BB8
:1014D00022689A4285B007D003F02AFD044620BB5B
:1014E0000024204605B030BD254B627D25481A708A
:1014F000237D03724FF48073C0F8F8314FF400730A
:10150000C0F80C3300254FF44073C0F820341E4956
:10151000C0F8E450C922093000F008FB2046E02260
:10152000294600F015FB0124DBE7184A184D136C1F
:1015300043F000731364AA6D164B9A42D0D12B6E00
:10154000013B7E2BCCD8144A07CA01AB83E80700C5
:101550001846032100F06CFD6B6D83424FF00003D1
:10156000BED12A6D8A4201BFAB65054B2A6E1A7047
:1015700003BF0A4BEA6D1A601C46B2E79AAD44C538
:10158000BC2400209856002016000020003802409D
:10159000006600405041A0B0586600401023002073
:1015A00037B500F077FD1D4D1D4C288102232168C1
:1015B0001C486B71012201F077FB1B48216850F831
:1015C000D03F01225B68984700230193174B1849CD
:1015D00000931848184B4FF4805201F0D5FF174B79
:1015E000197811B1134801F0F7FF01F0D9FC044656
:1015F000FFF7C6FB4FF4C873B0FBF3F202FB130313
:1016000004F5167010FA83F00D4B186003F086FC99
:1016100008B10F232B8103B030BD00BFB0240020E0
:1016200010230020F8340020F8440020B1100008F6
:10163000C0240020C8340020C1110008BC240020B0
:10164000C43400202DE9F04F2DED028BDFF85082DD
:1016500093B00BAF9FED838BFFF7D0FC00230A9371
:10166000ADF834300B937B600025844CDFF810A27A
:101670002E4601238DF81C3023688DED008B4FF032
:10168000000BD3F808908DF81DB05B460DF11D02DC
:1016900007A92046C8479DF81C90B9F1000F24D037
:1016A000D8F8143083F40043C8F814301022594697
:1016B0000EA800F04DFA236808AA5E690AA90DF188
:1016C0001E032046B04797E803000FAB83E80300F2
:1016D0009DF834308DF844300A9B0E930EA9DDE955
:1016E0000823504602F032FA4E4605F2344540F6E1
:1016F000680304F586549D4204F11004B9D1002E0C
:10170000B2D15F4801F070FF002840D15D4D01F07B
:1017100047FC2B6898423AD301F042FC0446FFF79D
:101720002FFB4FF4C873B0FBF3F202FB130304F575
:10173000167010FA83F02860534D8DF828602E78CB
:1017400016B901238DF82830C6F11004E4B20EA8B2
:10175000FFF72EFB062C28BF06240EAB2246991954
:101760000DF1290000F0E2F90AAB0393182302936C
:101770000134464B0193E4B20123009340480494A2
:101780003AA3D3E9002301F075FF00232B7001F089
:1017900007FC3F4A3F4C1368C31AB3F57A7F2FD337
:1017A000106001F0FFFB02460B46354801F0FAFFDE
:1017B000334801F019FF18B3237A374D002B14BFBB
:1017C000032302236B7101F0EBFB0EAE4FF47A732F
:1017D0000122B0FBF3F031462860284600F0DAFA27
:1017E000182302932D4B019380B240F25513CDE99B
:1017F0000360009322481FA3D3E9002301F03AFFBE
:10180000237A93B101F0CCFB002506464FF48A778A
:1018100094F8D900284400F0030007FB004393F834
:10182000E82072B10135042DF2D1C82003F002F88E
:10183000237A002B7FF40DAF13B0BDEC028BBDE813
:10184000F08FD3F8E02042B12368FA2B38BFFA2397
:10185000B21A0533B2EB430FE4D3FFF77FFB002846
:10186000E0D1E2E70000000000000000401DA120E0
:1018700026812A0BF1C6A7C1D068080FF8340020D2
:10188000C8340020C4340020C1340020C0340020FB
:10189000C85B002098560020B0240020CC5B0020BC
:1018A0000004024008B5064800F074FF054800F047
:1018B00071FFBDE80840044A0449002003F05CBE03
:1018C000F8340020C8450020205C00207D1100086D
:1018D0007047000070B5104B1B780133DBB2012B51
:1018E0000C4612D80D4B1D6829684FF47A730E6AA6
:1018F000A2FB0332014622462846B047844204D167
:10190000074B00221A70012070BD4FF4FA7002F0EC
:1019100091FF0020F8E700BF1C23002020230020B7
:10192000105C002007B50023024601210DF10700DD
:101930008DF80730FFF7CEFF20B19DF8070003B008
:101940005DF804FB4FF0FF30F9E700000A4608B5E8
:101950000421FFF7BFFF80F00100C0B2404208BD84
:1019600030B4074B0A461978064B53F821402368D8
:10197000DD69054B0146AC46204630BC604700BFE0
:10198000105C002020230020A086010070B503F029
:1019900015F9094E094D30800024286833888342A8
:1019A00008D903F005F92B6804440133B4F5803FEE
:1019B0002B60F2D370BD00BF125C0020D05B002012
:1019C00003F0ACB900F1006000F5803000687047AA
:1019D00000F10060920000F5803003F035B900009E
:1019E000054B1A68054B1B889B1A834202D9104489
:1019F00003F0DEB800207047D05B0020125C0020AE
:101A0000024B1B68184403F0DBB800BFD05B00201A
:101A1000024B1B68184403F0EBB800BFD05B0020FA
:101A200010F003030AD1B0F5047F05D200F1005095
:101A3000A0F51040D0F80038184670470023FBE7A7
:101A400000F10050A0F51040D0F8100A70470000D7
:101A5000064991F8243033B10023086A81F8243014
:101A60000822FFF7B5BF0120704700BFD45B0020FC
:101A7000014B1868704700BF002004E070B5194B97
:101A80001D68194B0138C5F30B0408442D0C0422C2
:101A90001E88A6420BD15C680A46013C824213466E
:101AA0000FD214F9016F4EB102F8016BF6E7013A5B
:101AB00003F10803ECD181420B4602D22C2203F839
:101AC000012B0A4A05241688AE4204D1984284BFED
:101AD000967803F8016B013C02F10402F3D1581A25
:101AE00070BD00BF002004E0705700085C5700087C
:101AF000022802BF024B4FF000429A61704700BFBC
:101B000000040240022802BF024B4FF400429A61D7
:101B1000704700BF00040240022801BF024A536917
:101B200083F40043536170470004024010B5002362
:101B3000934203D0CC5CC4540133F9E710BD0000DC
:101B400003460246D01A12F9011B0029FAD1704748
:101B500002440346934202D003F8011BFAE77047A0
:101B60002DE9F8431F4D144695F824200746884672
:101B700052BBDFF870909CB395F824302BB920222B
:101B8000FF2148462F62FFF7E3FF95F82400C0F1DC
:101B90000802A24228BF2246D6B24146920005EB77
:101BA0008000FFF7C3FF95F82430A41B1E44F6B253
:101BB000082E17449044E4B285F82460DBD1FFF787
:101BC00047FF0028D7D108E02B6A03EB820383424A
:101BD000CFD0FFF73DFF0028CBD10020BDE8F88330
:101BE0000120FBE7D45B0020024B1A78024B1A70ED
:101BF000704700BF105C00201C23002003494FF4F5
:101C000061430B60024B186802F0DABCFC5B0020F9
:101C100020230020094B10B5142204460021184649
:101C2000FFF796FF064A074B127804600146BDE8AD
:101C3000104053F8220002F0C3BC00BFFC5B002040
:101C4000105C0020202300202DE9F0470D460446BB
:101C500000219046284640F27912FFF779FF23468B
:101C600020220021284601F013FF231D02222021FB
:101C7000284601F00DFF631D03222221284601F0B2
:101C800007FFA31D03222521284601F001FF04F1CF
:101C9000080310222821284601F0FAFE04F110035F
:101CA00008223821284601F0F3FE04F1110308222E
:101CB0004021284601F0ECFE04F1120308224821DD
:101CC000284601F0E5FE04F11403202250212846A5
:101CD00001F0DEFE04F1180340227021284601F0D5
:101CE000D7FE04F120030822B021284601F0D0FEDF
:101CF00004F121030822B821284601F0C9FE04F1AD
:101D00002207C0263B46314608222846083601F005
:101D1000BFFEB6F5A07F07F10107F3D104F132034E
:101D200008223146284601F0B3FE002704F1330AA9
:101D300094F832304FEAC7099F4209F5A47615D3CB
:101D4000B8F1000F08D1314604F5997307222846EF
:101D500001F09EFE09F24F16274694F832213B1BF4
:101D600093420CD3F01DC008BDE8F0870AEB0703CF
:101D700008223146284601F08BFE0137D8E707F2EA
:101D8000331331460822284601F082FE0836013717
:101D9000E3E7000013B5044608460021016023462E
:101DA000C0F803102022019001F072FE0198231D5B
:101DB0000222202101F06CFE0198631D03222221E2
:101DC00001F066FE0198A31D0322252101F060FEAB
:101DD000019804F108031022282101F059FE072080
:101DE00002B010BDF7B50023047F00910E46072214
:101DF0001946054601F010FD731C009301220023D3
:101E00000721284601F008FDC4B9B31C0093052240
:101E100023460821284601F0FFFC0D243746B278FE
:101E2000BB1B934211D32B7FA88A0734E408BBB9AC
:101E3000844294BF0020012003B0F0BDAB8ADB00D8
:101E4000083BDB08B3700824E8E7FB1C009321463D
:101E500000230822284601F0DFFC08340137DEE7C2
:101E6000201A18BF0120E7E7F7B50023047F00918F
:101E70000E4608221946054601F0CEFC731CC4B973
:101E80000822009311462346284601F0C5FC102481
:101E9000012372785F1C013B934211D32B7FA88AE8
:101EA0000734E408BBB9844294BF0020012003B08A
:101EB000F0BDAB8ADB00083BDB0873700824E7E762
:101EC000F3190093214600230822284601F0A4FCC0
:101ED00008343B46DDE7201A18BF0120E7E7000081
:101EE000F8B50E4605461446002181223046FFF71C
:101EF0002FFE2B4608220021304601F0C9FD7CB997
:101F00006B1C07220821304601F0C2FD0F2401237B
:101F10006A785F1C013B934204D3E01DC008F8BD02
:101F20000824F4E7EB1921460822304601F0B0FD01
:101F300008343B46ECE70000F8B50E46054614466B
:101F40000021CE223046FFF703FE2B462822002137
:101F5000304601F09DFD7CB905F1080308222821D7
:101F6000304601F095FD30242F462A7A7B1B9342A0
:101F700004D3E01DC008F8BD2824F5E707F10903E4
:101F800021460822304601F083FD08340137ECE792
:101F9000F7B5047F00910E4601231022002105466B
:101FA00001F03AFCC4B9B31C009309222346102166
:101FB000284601F031FC192437467288BB1B9A422F
:101FC00011D82B7FA88A0734E408BBB9844294BF98
:101FD0000020012003B0F0BDAB8ADB00103BDB0822
:101FE00073801024E8E73B1D00932146002308225C
:101FF000284601F011FC08340137DEE7201A18BF2B
:102000000120E7E730B5094D0A4491420DD011F89F
:10201000013B5840082340F30004013B2C4013F0DF
:10202000FF0384EA5000F6D1EFE730BD2083B8ED1E
:10203000F7B54FF0FF33DFF854C0DFF854E000EBA2
:1020400081011A4688421CD050F8044B019401AF1C
:10205000042417F8015B82EA05620825DB1816469E
:1020600005F1FF355241002EBCBF83EA0C0382EA22
:102070000E0215F0FF05F1D1013C14F0FF04E8D188
:10208000E0E7D843D14303B0F0BD00BF9336EAA9DF
:10209000EBE1F042F7B5384A106851686B4603C36C
:1020A0006A4636493648082303F0C6FA0446002833
:1020B00033D10A25334A106851686B4603C36A4618
:1020C00031492F48082303F0B7FA0446002849D0C5
:1020D0000369B3F5E02F45D8B0F8661040F20B4223
:1020E00091423FD1294A024402F15C018B4239D32B
:1020F0005C3B234900209E1AFFF784FF32460746C7
:1021000004F164010020FFF77DFFA3689F4229D1FD
:10211000E368984208BF002524E00369B3F5E02F87
:1021200027D8418B40F20B42914220D1174A0244FA
:1021300002F110018B4218D3103B114900209D1A67
:10214000FFF760FF2A46064604F118010020FFF75A
:1021500059FFA3689E4202D1E368984201D00D2541
:10216000A8E70025284603B0F0BD1025A2E70C25FE
:10217000A0E70B259EE700BF90570008DCFF060094
:10218000000001089957000890FF06000800FFF7BB
:1021900010B5037C044613B9006803F035FA2046F5
:1021A00010BD00000023BFF35B8FC360BFF35B8FE4
:1021B000BFF35B8F8360BFF35B8F7047BFF35B8FB1
:1021C0000068BFF35B8F704770B505460C30FFF7B2
:1021D000F5FF05F1080604463046FFF7EFFFA04281
:1021E00006D930466D68FFF7E9FF2544281A70BD0F
:1021F0003046FFF7E3FF201AF9E7000070B5054607
:10220000406898B105F10800FFF7D8FF05F10C060A
:1022100004463046FFF7D2FF8442304694BF6D68D3
:102220000025FFF7CBFF013C2C44201A70BD0000B5
:1022300038B50C460546FFF7C7FFA04210D305F19D
:102240000800FFF7BBFF04446868B4FBF0F100FB33
:102250001144BFF35B8F0120AC60BFF35B8F38BDCF
:102260000020FCE72DE9F041144607460D46FFF734
:10227000C5FF844228BF0446D4B1B84658F80C6B59
:102280004046FFF79BFF3044286040467E68FFF7DA
:1022900095FF331A9C4203D86C600120BDE8F081A1
:1022A0006B60A41B3B68AB602044E8600220F5E74C
:1022B0002046F3E738B50C460546FFF79FFFA042DE
:1022C00010D305F10C00FFF779FF04446868B4FBF4
:1022D000F0F100FB1144BFF35B8F0120EC60BFF312
:1022E0005B8F38BD0020FCE72DE9FF418846694639
:1022F0000746FFF7B7FF6C4606B204EBC60600259B
:10230000B44209D06268206808EB0501FFF70EFCB3
:10231000636808341D44F3E729463846FFF7CAFFCF
:10232000284604B0BDE8F081F8B505460C300F46EC
:10233000FFF744FF05F1080604463046FFF73EFF6D
:10234000A042304688BF6C68FFF738FF201A38601B
:1023500020B130462C68FFF731FF2044F8BD000063
:1023600073B5144606460D46FFF72EFF844228BF7C
:1023700004460190DCB101A93046FFF7D5FF019B6F
:1023800033B93268C5E90233C5E9002401200CE005
:102390009C4238BF01942860019868608442F5D956
:1023A0003368AB60241AEC60022002B070BD204696
:1023B000FBE700002DE9FF410F466946FFF7D0FF1C
:1023C0006C4600B204EBC0050026AC4209D0D4F83C
:1023D000048054F8081BB8194246FFF7A7FB46448F
:1023E000F3E7304604B0BDE8F081000038B505469B
:1023F000FFF7E0FF044601462846FFF719FF204695
:1024000038BD0000302383F3118862B670470000A6
:10241000002383F3118862B67047000010B402688D
:1024200054681A4623465DF8044B1847012070474C
:102430000020704700207047704700000020704760
:102440000E20704700F5805090F8C800C0F340009F
:102450007047000000F5805090F9C90070470000F7
:10246000F7B50C68BDF8207014F000541E466FD10B
:102470000B7B082B6CD8FFF7C5FF4569AB685B0188
:102480000CD4AB681B0108D4AC6814F080545DD147
:10249000FFF7BEFF204603B0F0BD01240B6804F136
:1024A000180C002BB8BFDB004FEA0C1CB4BF43F084
:1024B00004035B0545F80C300B680FFA84FC13F03D
:1024C000804F18BF05EB0C1E05EB0C1C1EBFDEF881
:1024D000803143F00203CEF880310B7BCCF884319D
:1024E00005EB04158B68C5F88C314B68C5F888314D
:1024F000DCF8803143F00103CCF8803100EB441567
:1025000041F268031D4403EB44130344C5E900266C
:1025100008330D4601F10C0C55F804EB43F804EBBD
:102520006545F9D184342D881D8000EB441407F0F3
:102530000303257925F00B052B432371FFF768FF73
:102540000097334600F04EFD0120A4E70224A5E7E2
:102550004FF0FF309FE7000013B500F58054019164
:10256000E06DFFF74BFE1F280AD90199E06D20228C
:10257000FFF7BAFEA0F120035842584102B010BD47
:102580000020FBE708B500F58050FFF73BFFC06D6A
:10259000FFF708FEBDE80840FFF73ABF00220260DF
:1025A000828142608260704710B500220023C0E93A
:1025B00000230023044603810C30FFF7EFFF204681
:1025C00010BD0000F0B5054600F580500C4690F8AF
:1025D000C83013F0040FC3F3800108BF114661F344
:1025E000820304F1840680F8C83005EB461389B0F5
:1025F0001B79D8072ED57AB319072DD46846FFF773
:10260000D3FF05EB441303F5835303F1180703AA23
:10261000103318685968144603C40833BB42224675
:10262000F7D1186820609B88A380DDE90E23CDE9EF
:1026300000230123ADF808302B686946DB6B284680
:10264000984705EB46152B791A075CBF43F0080342
:102650002B7101E0002AF4D109B0F0BD2DE9F0475B
:10266000074688B007F5805468469A468846FFF7C3
:10267000C9FE9146FFF798FFE06DFFF7A5FD1F2803
:1026800029D9E06D20226946FFF7B0FE202822D12B
:1026900003AD444605AB2E4603CE9E4220606160EA
:1026A000354604F10804F6D130682060B388A38071
:1026B000DDE90023C9E90023BDF80830AAF800309D
:1026C000FFF7A6FE4A4653464146384608B0BDE8E5
:1026D000F04700F075BCFFF79BFE002008B0BDE896
:1026E000F08700002DE9F84F0023C0E90133264BA5
:1026F000044640F8183B0F46FFF750FF04F128004E
:10270000FFF752FF04F1480804F5825546460835A4
:1027100030462036FFF748FFAE42F9D104F5805528
:102720004FF480534FF00009C5E91339C5F84880CC
:102730000123EE6504F5875804F58456C5F85490D6
:1027400085F8583085F86030083608F108084FF0F1
:10275000000A4FF0000B46E908ABA6F11800FFF79E
:102760001DFF203646F8289C4645F4D1012F85F8F8
:10277000C97002D9054800F00DFC054B53F827300D
:1027800063612046BDE8F88FDC570008A4570008B5
:10279000C057000810B5044B197804464A1C1A703B
:1027A000FFF7A0FF204610BD1C5C00202DE9F0477C
:1027B000002950D0294B2A4FB7FBF1F599428CBF25
:1027C0000A231123581EB5FBF3FC03FB1C53C4B2B0
:1027D0002BB102280346F5D80020BDE8F0870CF1A4
:1027E000FF36B6F5806FF7D2C4EBC40E0EF10303CB
:1027F0004FEAE309C3F3C703A4EB030809F1010A95
:102800004FF47A755FFA88F009FB05555AFA88F893
:10281000B5FBF8F5B5F5617FC1BF0EF1FF33C3F32A
:10282000C703E01AC0B25C1C50FA84F40CFB04F439
:10283000B7FBF4F4A142CFD1013BDBB20F2BCBD8D5
:102840000138C0B20728C7D80021107116809170D6
:10285000D3700120C1E70846BFE700BF3F420F0029
:1028600040787D0170B505460E464FF47A746B6969
:102870005B6803F00103B34207D04FF47A7001F0B4
:10288000D9FF013CF3D1204670BD0120FCE70000D8
:1028900030B54269936913F0700F16D000230B4CCA
:1028A000936103F1840200EB421211794D0709D5BF
:1028B000890707D5416954F823508D60117941F09B
:1028C000040111710133032BEBD130BDC85700084F
:1028D00073B51D46436916469A68D207044609D562
:1028E0009A6801219960C2F34002CDE90065002198
:1028F000FFF768FE63699A68D1050BD59A684FF4B3
:1029000080719960C2F34022CDE900650121204623
:10291000FFF758FE63699A68D2030BD59A684FF4A3
:1029200080319960C2F34042CDE900650221204622
:10293000FFF748FE204602B0BDE87040FFF7A8BF91
:102940000C4B10B51C561B5C012B11D800F02AFB58
:1029500050EA0103024602D0421E61F10001064B1B
:1029600053F8240020B1BDE810400B46FFF7B0BF7C
:1029700010BD00BFBC570008145C0020F8B5044629
:10298000466900296CD106F10C07386880076AD0C7
:1029900006EB01153868D5F8B00110F0040FD5F832
:1029A000B0011ABFC00840F00040400DA061D5F84A
:1029B000B0C11CF0020F1CBF40F08040A061D5F8F0
:1029C000B40106EB011100F00F0084F82400D1F8E7
:1029D000B8012077D1F8B801000A6077D1F8B801C2
:1029E000000CA077D1F8B801000EE077D1F8BC0157
:1029F00084F82000D1F8BC01000A84F82100D1F845
:102A0000BC01000C84F82200D1F8BC11090E84F836
:102A100023103821396004F1340004F1180104F165
:102A2000240551F8046B40F8046BA942F9D10988D8
:102A30000180C4E90A2321460023238651F8283B5C
:102A40002046DB6B984704F58052204692F8C83048
:102A500043F0040382F8C830BDE8F840FFF718BF20
:102A600006F1100791E7F8BD0D4B70B51D561B5CC4
:102A7000012B0C4612D800F095FA02460B4652EA9A
:102A8000030102D0013A63F10003064951F8250021
:102A900020B12146BDE87040FFF770BF70BD00BF98
:102AA000BC570008145C0020F8B500F583511E46A1
:102AB000FFF7A8FCDFF844C00831002404F18405C6
:102AC00000EB45152B795F070ED4DB060CD5D1E959
:102AD00000739742B34107D243695CF824709F604A
:102AE0002B7943F004032B710134032C01F12001F5
:102AF000E4D1BDE8F840FFF78BBC00BFC857000821
:102B000008B5FFF77FFCFFF7C3FEBDE80840FFF7FD
:102B10007FBC0000F8B543690546986800F0E050B6
:102B2000B0F1E05F0F461FD0E8B1FFF76BFC05F591
:102B300083541034002606F1840305EB43131B79FC
:102B40001A0706D50136032E04F12004F3D1012023
:102B500007E05B07F6D42146384600F07DFA0028EE
:102B6000F0D1FFF755FCF8BD0120FCE700F58050DF
:102B700008B5FFF747FCC06DFFF726FBFFF748FCE1
:102B800043090CBF0120002008BD0000F8B51D4618
:102B9000002313700F4606461446FFF7E7FF80F048
:102BA0000100387025B129463046FFF7B3FF207089
:102BB000F8BD00002DE9B8410C4615461F46804679
:102BC00000F0F0F90B462178024609B9287850B197
:102BD0004046FFF769FFFFF793FF3B462A46214631
:102BE000FFF7D4FF0120BDE8B881000038B500F53B
:102BF0008054FFF707FC2A4D94F8C930EB5CDBB139
:102C0000012B27D0FFF704FC94F8C830DB0746D42B
:102C1000002944D0FFF7F6FB94F8C930EB5C33B3DE
:102C2000012B31D094F8C83043F0010384F8C83048
:102C3000BDE83840FFF7ECBB1A4B1A6C42F000724B
:102C40001A641A6A42F000721A621A6A22F000725A
:102C50001A62D7E7134B1A6C42F080621A641A6A40
:102C600042F080621A621A6A22F08062F0E7032161
:102C7000132001F0D9FA0321142001F0D5FA032121
:102C8000152001F0D1FACDE703213F2001F0CCFA65
:102C90000321402001F0C8FA03214120F1E738BDAB
:102CA000B8570008003802402DE9F04700F580557C
:102CB00088B095F8C930022B0446884616467FD85E
:102CC000844F57F823200AB947F82300D7F800A00B
:102CD000C4F80C802674BAF1000F63D095F8C9309F
:102CE000012B6FD001212046FFF780FFFFF78AFB01
:102CF0006269136823F0020313606269136843F08A
:102D000001031360636900275F6101212046FFF71B
:102D10007FFBFFF7A7FD002800F09580E86DFFF727
:102D200041FA04F58359BA4609F108092022002125
:102D30006846FEF70DFF02A8FFF730FCCDF818A09B
:102D40006A4609EB07030DF1180E9446BCE8030030
:102D5000F44518605960624603F10803F5D1DCF8C8
:102D60000000186020379CF804201A71602FDDD114
:102D700095F8C8306FF38203002785F8C8306A469B
:102D800041462046ADF80070ADF802708DF8047031
:102D9000FFF70CFD636948BB4FF400421A6008B0AE
:102DA000BDE8F08741F2D00002F0EEFB814610B1A1
:102DB0005146FFF797FCC7F80090B9F1000F8DD18D
:102DC0000020ECE7386803681B6B98470146002831
:102DD00088D13868FFF70AFF3868036832465B68B5
:102DE0004146984700287FF47DAFE9E761221A60E9
:102DF0009DF802309DF803201B06120402F4702295
:102E000003F040731343BDF80020C2F309021343DB
:102E10009DF804201205022E02F4E0020CBF4FF0D0
:102E200000410021134362690B43D361636913229C
:102E30005A616269136823F0010313603946204622
:102E4000FFF710FD08B96369A6E795F8C930002BB4
:102E500039D16169D1F8002242F00102C1F80022A3
:102E60006169D1F8002222F47C5222F00E02C1F8EE
:102E700000226169D1F8002242F46062C1F80022A8
:102E80006269C2F814326269C2F8043262696FF092
:102E90007841C2F80C126269C2F840326269C2F825
:102EA00044326269C2F8B0326269C2F8B43263690E
:102EB00044F20102C3F81C226269D2F8003223F006
:102EC0000103C2F8003295F8C83043F0020385F8D8
:102ED000C83064E7145C002008B50020FFF730FD1F
:102EE000BDE8084001F082B808B500210846FFF7A8
:102EF000BBFDBDE8084001F079B8000008B501212C
:102F00000020FFF7B1FDBDE8084001F06FB80000F8
:102F100008B50120FFF714FDBDE8084001F066B8D0
:102F200008B500210120FFF79FFDBDE8084001F032
:102F30005DB8000008B501210846FFF795FDBDE822
:102F4000084001F053B8000000B59BB0EFF30981D1
:102F500068226846FEF7EAFDEFF30583014B9B6BA1
:102F6000FEE700BF00ED00E008B5FFF7EDFF000051
:102F700000B59BB0EFF3098168226846FEF7D6FDE5
:102F8000EFF30583014B5B6BFEE700BF00ED00E054
:102F9000FEE700000FB408B5029801F0E1FBFEE780
:102FA00001F008BF01F0E0BE13B56C4684E80600EE
:102FB000031D94E8030083E80500012002B010BD62
:102FC00073B58568019155B11B885B0707D4D0E9BB
:102FD00000369B6B9847019AC1B23046A847012042
:102FE00002B070BDF0B5866889B005460C465EB18A
:102FF000BDF838305B070AD4D0E900379B6B98479F
:103000002246C1B23846B047012009B0F0BD0022C7
:103010000023CDE900230023ADF808300A4603ABB6
:1030200001F10806106851681C4603C40832B24218
:103030002346F7D1106820609288A280FFF7B2FF84
:103040000423ADF808302B68CDE90001DB6B69463D
:1030500028469847D8E7000030B503680968DD0FB7
:10306000B5EBD17F23F0604421F060424FEAD1708C
:103070000BD0002BB8BFA40C0029B8BF920C94420F
:1030800002D034BF0120002030BD944205D1C1F3ED
:103090008070C3F380738342F6D194422CBF00202A
:1030A0000120F1E72DE9F041456A15B94162BDE81B
:1030B000F0814B6823F06047C3F38A464FEAD37E22
:1030C000C3F3807816EA230638BF3E46AC462B464B
:1030D0005A68BEEBD27F22F060440AD0002A18DA88
:1030E000A40CB44217D19D420FD10D60DEE7134608
:1030F000EEE7A74207D102F08044C2F38072424556
:103100000BD054B1EFE708D2EDE7CCF800100B601C
:10311000CDE7B44201D0B442E5D81A689C46002AF3
:10312000E5D11960C3E700002DE9F047089D01F0E3
:1031300007044FEAD508224405F0070500EBD1004B
:103140004FF47F49944201D1BDE8F08704F00707AE
:1031500005F0070A57453E4638BF5646C6F10806F1
:10316000111B8E4228BF0E46E10808EBD50E415CCC
:1031700013F80EC0B94029FA06F721FA0AF1FFB296
:103180008CEA010147FA0AF739408CEA010C03F88E
:103190000EC034443544D5E780EA0120082341F2CB
:1031A000210201B24000002980B203F1FF33B8BF11
:1031B000504013F0FF03F4D17047000038B50C46BF
:1031C0008D18A54200D138BD14F8011BFFF7E4FFAC
:1031D000F7E7000042684AB1136843604389818978
:1031E00001339BB29942438138BF838110467047B7
:1031F00070B588B0202204460D4668460021FEF7CF
:10320000A7FC20460495FFF7E5FF024658B16B4640
:10321000054608AE1C4603CCB442286069602346CC
:1032200005F10805F6D1104608B070BD082817D979
:1032300009280CD00A280CD00B280CD00C280CD054
:103240000D280CD00E2814BF4020302070470C20D1
:1032500070471020704714207047182070472020B6
:1032600070470000082817D90C280CD910280CD951
:1032700014280CD918280CD920280CD930288CBF38
:103280000F200E207047092070470A2070470B203E
:1032900070470C2070470D20704700002DE9F8435F
:1032A000078C072F04461ED9D0E9029800254FF657
:1032B000FF73C5F12006A5F1200029FA05F108FAEF
:1032C00006F628FA00F031430143C9B21846FFF769
:1032D00063FF0835402D0346EBD1E1693A46BDE86E
:1032E000F843FFF76BBF4FF6FF70BDE8F8830000AF
:1032F00010B54B6823B9CA8A63F30902CA8210BDAC
:1033000004691A681C600361C38A013BC3824A6076
:10331000EFE700002DE9F84F1D46CB8A0F46C3F3B7
:1033200009010529814692460B4630D00020AAB2F9
:1033300007F11A049EB2042E1FFA80F80FD89045A8
:1033400003F1010306D3FB8A0A4462F30903FB82FB
:1033500001201AE01AF80060E6540130EAE79045CF
:10336000F1D2A1F1050B1C237C68BBFBF3F203FB3C
:1033700012BB1FFA8BF6002C45D14846FFF72AFFF7
:10338000044638B978606FF00200BDE8F88F4FF05E
:103390000008E6E7002606607860ADB24FF0000B4B
:1033A000454510D90AEB0803221D13F8011B91555E
:1033B000B1B208F101081B291FFA88F82BD0454546
:1033C00006F10106F1D8FB8AC3F30902154465F33F
:1033D0000903BCE7013292B21C462368002BF9D1E5
:1033E0006B1F0B441C21B3FBF1F301339BB29A42D8
:1033F000D3D2BBF1000FD0D14846FFF7EBFE20B986
:10340000C4F800B0BFE70122E7E7C0F800B05E46AD
:1034100020600446C1E74545D5D94846FFF7DAFEA6
:1034200008B92060AFE7C0F800B00026206004466D
:10343000B6E700002DE9F04F2DED028B1C4683B05E
:103440005B69019207468846002B00F09A80238C26
:103450002BB1E269002A00F09480072B35D807F1E0
:103460000C00FFF7B7FE054638B96FF00205284695
:1034700003B0BDEC028BBDE8F08F14220021FEF7F3
:1034800067FB228CE16905F10800FEF74FFB208CF9
:10349000013080B2FFF7E6FEFFF7C8FE013880B2C8
:1034A0002084013028746369228C1B782A4403F03D
:1034B0001F0363F03F0348F0004113723846696010
:1034C0002946FFF7EFFD0125D1E700F10C034FF08E
:1034D000000908EE103A4FF0800A4E464D4618EEAD
:1034E000100AFFF777FE83460028BED01422002181
:1034F000FEF72EFB002E3AD1019BABF808300222DA
:103500000BF1080E1FFA82FC0CF10100BCF1060F52
:10351000218C80B201D88E422BD3FFF7A3FEFFF798
:1035200085FE62691278013802F01F028E4208BFE0
:103530004FF0400A42EA49121BFA80F14AEA020AB5
:10354000013048F0004281F808A08BF81000CBF859
:10355000042059463846FFF7A5FD238C0135B342B8
:103560002DB289F001094FF0000AB8D17FE700229F
:10357000C6E7E169895D0EF802100136B6B2013284
:10358000C0E76FF0010572E7F8B515460E46302228
:10359000002104461F46FEF7DBFA069B6360B5F583
:1035A000001F079BA76034BF6A094FF6FF72A36232
:1035B00097B2E66104F1100000239A4206D8002376
:1035C0000360A782E3822383E360F8BD06600133D2
:1035D00030462036F1E7000003781BB94BB2002BD0
:1035E000C8BF01707047000000787047F8B50C46FE
:1035F000C969074611B9238C002B37D1257E1F2DB1
:1036000034D8387828BB228C072A2CD8268A36F062
:1036100003032BD14FF6FF70FFF7D0FD20F0010020
:103620003102400441EA0561400C41EA40254FF671
:10363000FF72234629463846FFF7FCFE002807DDC7
:10364000626913780133DBB21F2B88BF002313702C
:10365000F8BD218A2D0645EA012505432046FFF7DE
:103660001DFE0246E5E76FF00300F1E76FF0010091
:10367000EEE7000070B58AB0044616460021282205
:1036800068461D46FEF764FABDF83830ADF81030D4
:103690000F9B05939DF840308DF81830119B0793D0
:1036A0006946BDF84830ADF820302046CDE90265C6
:1036B000FFF79CFF0AB070BD2DE9F041D3690546C4
:1036C0000C4616460BB9138C5BBB377E1F2F28D8D0
:1036D00095F80080B8F1000F26D03046FFF7DEFDE8
:1036E0003378210241EAC33141EA0801338A41EAD1
:1036F000076141EA03410246334641F08001284612
:10370000FFF798FE00280ADD3378012B07D1726994
:1037100013780133DBB21F2B88BF00231370BDE881
:10372000F0816FF00100FAE76FF00300F7E70000A7
:10373000F0B58BB004460D46174600212822684696
:103740001E46FEF705FA9DF84C305A1E534253416F
:103750008DF800309DF84030ADF81030119B059386
:103760009DF848308DF81830149B07936A46BDF8D1
:103770005430ADF8203029462046CDE90276FFF7D7
:103780009BFF0BB0F0BD0000406A00B104307047F1
:10379000436A1A68426202691A600361C38A013B84
:1037A000C38270472DE9F041D0F82080194E1446AD
:1037B0001D464146002709B9BDE8F081D1E9022341
:1037C000A21A65EB0303964277EB03031ED2036A4A
:1037D0008B420DD1FFF78CFD036A1B6803620369FE
:1037E0000B60C38A0161016A013BC3828846E2E73C
:1037F000FFF77EFD0B68C8F8003003690B60C38AD1
:103800000161013BC382D8F80010D4E788460968FB
:10381000D1E700BF80841E002DE9F04F8BB00D462C
:10382000DDF8509014469B468046002800F0198130
:10383000B9F1000F00F01581531E3F2B00F21181EA
:10384000012A03D1BBF1000F40F00B810023CDE929
:103850000833B8F81430B5EBC30F4FEAC30703D3EE
:1038600000200BB0BDE8F08F2B199F42D8F80C3028
:103870003ABF7F1BFFB227461BB9D8F81030002B88
:103880007AD0272D4ED8C5F12806B7424FF0000355
:103890002CBFF6B23E4600932946D8F8080008AB84
:1038A0003246FFF741FCA7EB060A35445FFA8AFA75
:1038B000B8F8143003F10053053BDB000493D8F84B
:1038C0000C3003932821039B13B1BAF1000F2CD1C4
:1038D000D8F8100040B1BAF1000F05D0009608AB3F
:1038E0005246691AFFF720FC38B2002FB8D066079D
:1038F0000AD00AAB03EBD401624211F8083C02F093
:103900000702134101F8083C082C3CD9102C40F266
:10391000B580202C40F2B780BBF1000F00F09C80F6
:10392000082334E0BA460026C2E7049BE02B28BFF8
:10393000E02306930B44AB42059314D95A1B03981A
:103940000096924534BF5246D2B2691A08AB043091
:103950000792FFF7E9FB079A1644AAEB020A1544FF
:10396000F6B25FFA8AFA049B069A05999B1A0493A9
:10397000039B1B680393A6E70093D8F8080008ABE5
:103980003A462946AEE7BBF1000F13D00123B4EB52
:10399000C30F6CD0082C12D89DF82030621E23FA79
:1039A00002F2D50706D54FF0FF3202FA04F42343A2
:1039B0008DF820309DF8203089F8003051E7102C28
:1039C00012D8BDF82030621E23FA02F2D10706D5C4
:1039D0004FF0FF3202FA04F42343ADF82030BDF873
:1039E0002030A9F800303CE7202C0FD80899631E3E
:1039F00021FA03F3DA0705D54FF0FF3202FA04F497
:103A00000C430894089BC9F800302AE7402C2BD0BF
:103A1000DDE90865611EC4F12102A4F1210326FA43
:103A200001F105FA02F225FA03F311431943CB071A
:103A300012D50122A4F12003C4F1200102FA03F3FC
:103A400022FA01F1A240524243EA010363EB43032D
:103A500032432B43CDE90823DDE90823C9E90023DC
:103A6000FFE66FF00100FCE66FF00800F9E6082CB5
:103A7000A0D9102CB3D9202CEED8C3E7BBF1000F8E
:103A8000ADD0022383E7BBF1000FBBD004237EE758
:103A900030B5012A144638BF0124402C85B028BF18
:103AA00040240025012ACDE9025518D81B788DF84D
:103AB000083063070AD004AB03EBD405624215F863
:103AC000083C02F00702934005F8083C00910346C9
:103AD0002246002102A8FFF727FB05B030BD082AC7
:103AE000E4D9102A03D81B88ADF80830E1E7202A72
:103AF0008DBFD3E900231B680293CDE90223D8E7E9
:103B000010B5CB681BB98B600B618B8210BD04694B
:103B10001A681C600361C38A013BC382CA60F0E774
:103B200003064CBFC0F3C0300220704708B5024600
:103B3000FFF7F6FF022806D15306C2F30F2001D18A
:103B400000F0030008BDC2F30740FBE72DE9F04F8A
:103B500093B0CDE903230A6804461046FFF7E0FF5F
:103B6000022814BFC2F306260026002A0D4682460C
:103B700080F2F28112F0C04940F0EE81097B002909
:103B800000F0EA81022803D02378B34240F0E781B5
:103B9000C2F304630693104602F07F030593FFF718
:103BA000C5FF059B29444FEA834848EA0A4848EA8A
:103BB0004668CE7800230022CDE90823F309834626
:103BC00048EA0008029367D0059B009302466768A5
:103BD000534608A92046B847002800F0C381276A49
:103BE0004FB9414604F10C00FFF702FB074690B9BC
:103BF0006FF0020054E03B6998450DD03F68002FFC
:103C0000F9D1414604F10C00FFF7F2FA074600280B
:103C1000EED0236A3B60276297F817C006F01F08B2
:103C2000CCF3840CACEB08001FFA80FE0028B8BF70
:103C30000EF12000A8EB0C031FFA83FED7E9022146
:103C4000B8BF00B2002B0793BEBF0EF120031BB21A
:103C5000079352EA010338D0039BDFF824E39A1A52
:103C6000049B4FF0000C63EB010196457CEB0103D4
:103C70002BD36B7B97F81AE0734519D1029B002B6D
:103C800078D0012821DC7868F8B9DFF8F0C29445D3
:103C900070EB010316D337E0276A27B96FF00C00E9
:103CA00013B0BDE8F08F3B699845B5D03F68F4E7A5
:103CB000B24890427CEB010301D30020F0E7029B65
:103CC000002BFAD0079B0F2B17DCFA7DB30002F014
:103CD000030203F07C031343FB7539462046FFF7CC
:103CE00007FB6B7BBB76029B3BB9FB7DC3F3840276
:103CF000013262F38603FB75D0E76A7BBB7E9A4292
:103D0000DBD1029B002B35D0B309022B32D0039BB1
:103D1000BB60049BFB60142200210DA8FDF718FF77
:103D2000039B0A93049B0B932B1D0C932B7BADF8E9
:103D30003EB0013BDBB2ADF83C30069B8DF8423023
:103D4000059B8DF8433094F82C308DF840A083F01B
:103D500001038DF844308DF84180A3680AA92046FC
:103D60009847FB7DC3F38403013303F01F039B02D9
:103D7000FB82A2E7FB7DC6F34012B2EBD31F40F0FB
:103D8000F480C3F38403434540F0F280029A2B7B16
:103D9000B609002A4DD0F2075DD4032B40F2EB8028
:103DA000039BBB60049BFB602B7BAE1D033BDBB224
:103DB0003246394604F10C00FFF7ACFA00280CDA61
:103DC00039462046FFF794FAFB7DC3F384030133A1
:103DD00003F01F039B02FB820AE7DDE90884AB883E
:103DE0003B834FF6FF73C9F12000A9F1200228FAA6
:103DF00009F104FA00F0014324FA02F211431846D3
:103E0000C9B2FFF7C9F909F10809B9F1400F034632
:103E1000E9D1B8822A7B033AD2B23146FFF7CEF914
:103E2000FB7DB882DA43C2F3C01262F3C713FB759D
:103E300043E786B92E1D013BDBB23246394604F119
:103E40000C00FFF767FA0028BADB2A7BB88A013A30
:103E5000D2B23146E2E7F98AC1F30901013B0429F4
:103E6000DAB25BD8281D002307F11B069A4208D955
:103E700010F801CB06F801C0013101330529DBB28E
:103E8000F4D103990A9104990B91934207F11B0114
:103E90000C9138BF043379680D9134BF55FA83F320
:103EA00000230E93FB8AADF83EB0C3F309031A4416
:103EB000069B8DF84230059B8DF8433094F82C30EA
:103EC000ADF83C2083F001038DF8443000238DF8D9
:103ED00040A08DF841807B602A7BB88A013A291D79
:103EE000FFF76CF93B8BB882834203D1A3680AA920
:103EF0002046984720460AA9FFF702FEFB7DBA8AB2
:103F0000C3F38403013303F01F039B02FB823B8B4B
:103F10009A420CBF00206FF01000C1E67B68002BB6
:103F2000AFD0052001E01C3033461E68002EFAD1C8
:103F3000091A081D2E1D184401EB090CBCF11B0FBA
:103F40005FFA89F39DD89A429BD916F8013B00F895
:103F5000013B09F10109EFE76FF00900A0E66FF0FE
:103F60000A009DE66FF00B009AE66FF00D0097E6F1
:103F70006FF00E0094E66FF00F0091E640420F00E4
:103F800080841E00EFF3098305494A6B22F0010289
:103F90004A63683383F30988002383F311887047E9
:103FA00000EF00E0302080F3118862B60C4B0D4A20
:103FB000D96821F4E0610904090C0A43DA60D3F8F6
:103FC000FC20094942F08072C3F8FC200A6842F0E4
:103FD00001020A602022DA7783F82200704700BFCE
:103FE00000ED00E00003FA05001000E010B53023FA
:103FF00083F311880E4B5B6813F4006314D0F1EE69
:10400000103AEFF30984683C4FF08073E361094B89
:10401000DB6B236684F3098800F060FB10B1064B6C
:10402000A36110BD054BFBE783F31188F9E700BFDF
:1040300000ED00E000EF00E043060008460600083F
:10404000026843681143016003B1184770470000DC
:10405000024AD36843F0C003D36070470044004075
:1040600010B5054C054A0021204600F087FA044AA5
:10407000044BC4E9972310BD245C00205140000884
:104080000044004040787D01234A037C002918BF8A
:104090000A46012B30B5C0F868220CD11F4B98425C
:1040A00009D11F4B196C41F400311964196E41F4A8
:1040B000003119661B6EB2F904501468D0F86032F2
:1040C000D0F85C12002D03EB5403B3FBF4F3BEBF36
:1040D00023F0070503F0070343EA450394888B6048
:1040E000D38843F040030B61138943F001034B6114
:1040F00044F4045343F02C03CB6004F4A054002395
:104100000B60B4F5806F0B684B680CBF7F23FF23F7
:1041100080F8643230BD00BF1C580008245C0020C9
:10412000003802402DE9F041D0F85C62F76833684E
:10413000DA0504469DB20DD5302383F311884FF480
:1041400080610430FFF77CFF6FF4807333600023DD
:1041500083F31188302383F3118804F1040815F0E8
:104160002F033AD183F31188380615D5290613D5C4
:10417000302383F3118804F1380000F07BF9002824
:104180004EDA0821201DFFF75BFF4FF67F733B409F
:10419000F360002383F311887A0616D56B0614D5D5
:1041A000302383F31188D4E913239A420AD1236C74
:1041B00043B127F040073F041021201D3F0CFFF7BB
:1041C0003FFFF760002383F31188D4F86822D36897
:1041D00043B3BDE8F041106918472B0714D015F020
:1041E000080F0CBF00214FF48071E80748BF41F071
:1041F0002001AA0748BF41F040016B0748BF41F0CA
:1042000080014046FFF71CFFAD06736805D594F8A2
:1042100064122046194000F0E1F93568ADB29EE71E
:104220007060B6E7BDE8F08100F1604303F56143DB
:104230000901C9B283F80013012200F01F039A405C
:1042400043099B0003F1604303F56143C3F88021F8
:104250001A607047F8B5154682680669AA420B468F
:10426000816938BF8568761AB54204460BD2184674
:104270002A46FDF75BFCA3692B44A361A3685B1B83
:10428000A3602846F8BD0CD918463246FDF74EFC0F
:10429000AF1BE1683A463044FDF748FCE3683B4415
:1042A000EBE718462A46FDF741FCE368E5E7000026
:1042B00083689342F7B51546044638BF8568D0E950
:1042C0000460361AB5420BD22A46FDF72FFC63690B
:1042D0002B446361A36828465B1BA36003B0F0BD59
:1042E0000DD932460191FDF721FC0199E068AF1B21
:1042F0003A463144FDF71AFCE3683B44E9E72A46B5
:10430000FDF714FCE368E4E710B50A440024C36138
:10431000029B8460C0E90000C0E90511C160026130
:10432000036210BD08B5D0E90532934201D182681D
:1043300082B98268013282605A1C42611970D0E9E8
:1043400004329A4224BFC3684361002100F08EFA10
:10435000002008BD4FF0FF30FBE7000070B53023B0
:1043600004460E4683F31188A568A5B1A368A26927
:10437000013BA360531CA36115782269934224BFBB
:10438000E368A361E3690BB120469847002383F3F8
:104390001188284607E03146204600F057FA0028E9
:1043A000E2DA85F3118870BD2DE9F74F04460E4619
:1043B00017469846D0F81C904FF0300A8AF31188BF
:1043C0004FF0000B154665B12A4631462046FFF7EF
:1043D00041FF034660B94146204600F037FA002805
:1043E000F1D0002383F31188781B03B0BDE8F08F70
:1043F000B9F1000F03D001902046C847019B8BF311
:104400001188ED1A1E448AF31188DCE7C0E9051112
:10441000C160C3611144009B8260C0E9000001617A
:1044200003627047F8B504460D461646302383F301
:104430001188A768A7B1A368013BA36063695A1CF0
:1044400062611D70D4E904329A4224BFE36863615B
:10445000E3690BB120469847002080F3118807E0FC
:104460003146204600F0F2F90028E2DA87F311889D
:10447000F8BD0000D0E905239A4210B501D1826849
:104480007AB98268013282605A1C82611C780369A1
:104490009A4224BFC3688361002100F0E7F92046F7
:1044A00010BD4FF0FF30FBE72DE9F74F04460E46F5
:1044B00017469846D0F81C904FF0300A8AF31188BE
:1044C0004FF0000B154665B12A4631462046FFF7EE
:1044D000EFFE034660B94146204600F0B7F90028D8
:1044E000F1D0002383F31188781B03B0BDE8F08F6F
:1044F000B9F1000F03D001902046C847019B8BF310
:104500001188ED1A1E448AF31188DCE702684368BB
:104510001143016003B11847704700001430FFF7E2
:1045200043BF00004FF0FF331430FFF73DBF0000E2
:104530003830FFF7B9BF00004FF0FF333830FFF7D6
:10454000B3BF00001430FFF709BF00004FF0FF3188
:104550001430FFF703BF00003830FFF763BF0000DF
:104560004FF0FF323830FFF75DBF0000012914BF64
:104570006FF0130000207047FFF772BD37B5154686
:104580000E4A026000224260C0E902220122044673
:1045900002740B46009000F15C014FF480721430FD
:1045A000FFF7B2FE00942B464FF4807204F5AE7113
:1045B00004F13800FFF72AFF03B030BD305800087F
:1045C00010B53023044683F31188FFF75DFD022305
:1045D0002374002080F3118810BD000038B5C36932
:1045E00004460D461BB904210844FFF78FFF2946F6
:1045F00004F11400FFF796FE002806DA201D4FF4A0
:104600000061BDE83840FFF781BF38BD0023037566
:10461000826803691B6899689142FBD25A680360FB
:104620004260106058607047002303758268036918
:104630001B6899689142FBD85A6803604260106019
:104640005860704708B50846302383F311880B7D06
:10465000032B05D0042B0DD02BB983F3118808BD93
:104660008B6900221A604FF0FF338361FFF7CEFFA2
:104670000023F2E7D1E9003213605A60F3E700004B
:10468000FFF7C4BF054BD9680875186802681A603F
:10469000536001220275D860FBF7BEBF905E002018
:1046A00030B50C4BDD684B1C87B004460FD02B4651
:1046B000094A684600F06CF92046FFF7E3FF009BCB
:1046C00013B1684600F06EF9A86907B030BDFFF776
:1046D000D9FFF9E7905E002045460008044B1A68B0
:1046E000DB6890689B68984294BF00200120704767
:1046F000905E0020084B10B51C68D86822681A60CC
:10470000536001222275DC60FFF78EFF01462046D0
:10471000BDE81040FBF780BF905E0020044B1A6894
:10472000DB6892689B689A4201D9FFF7E3BF704744
:10473000905E002038B5074C074908480123002542
:104740002370656000F03AFC0223237085F3118822
:1047500038BD00BFF86000205C580008905E002063
:1047600008B572B6044B186500F0ECFA00F0A0FB37
:10477000024B03221A70FEE7905E0020F8600020D2
:1047800000F046B9EFF3118020B9EFF30583302232
:1047900082F311887047000010B530B9EFF305843B
:1047A000C4F3080414B180F3118810BDFFF7B6FFFD
:1047B00084F31188F9E700008B60022308618B8283
:1047C000084670478368A3F1840243F8142C0269F9
:1047D00043F8442C426943F8402C094A43F8242CFE
:1047E000C26843F8182C022203F80C2C002203F8AC
:1047F0000B2C044A43F8102CA3F12000704700BF93
:1048000031060008905E002008B5FFF7DBFFBDE829
:104810000840FFF735BF0000024BDB6898610F20AE
:10482000FFF730BF905E0020302383F31188FFF73D
:10483000F3BF000008B50146302383F31188082038
:10484000FFF72EFF002383F3118808BD064BDB68BA
:1048500039B1426818605A60136043600420FFF762
:104860001FBF4FF0FF307047905E002003689842F2
:1048700006D01A680260506099611846FFF700BFC1
:104880007047000010B503689C68A2420CD85C68B1
:104890008A600B604C602160596099688A1A9A603E
:1048A0004FF0FF33836010BD1B68121BECE7000064
:1048B0000A2938BF0A2170B504460D460A26601938
:1048C00000F076FB00F062FB041BA54203D8751CC8
:1048D0002E460446F3E70A2E04D9BDE870400120B5
:1048E00000F0ACBB70BD0000F8B5144B0D46D961AB
:1048F00003F1100141600A2A1969826038BF0A2257
:10490000016048601861A818144600F043FB0A27AC
:1049100000F03CFB431BA342064606D37C1C28192F
:1049200000F046FB27463546F2E70A2F04D9BDE8DA
:10493000F840012000F082BBF8BD00BF905E00206F
:10494000F8B506460D4600F021FB0F4A134653F812
:10495000107F9F4206D12A4601463046BDE8F84006
:10496000FFF7C2BFD169BB68441A2C1928BF2C4677
:10497000A34202D92946FFF79BFF2246314603484E
:10498000BDE8F840FFF77EBF905E0020A05E0020EB
:1049900010B4C0E9032300235DF8044B4361FFF723
:1049A000CFBF000010B5194C236998420DD0D0E953
:1049B0000032816813605A609A680A449A60002342
:1049C00003604FF0FF33A36110BD2346026843F834
:1049D000102F53600022026022699A4203D1BDE881
:1049E000104000F0DFBA936881680B44936000F0D8
:1049F000CDFA2269E1699268441AA242E4D91144CD
:104A0000BDE81040091AFFF753BF00BF905E0020B9
:104A10002DE9F047DFF8BC8008F110072C4ED8F8DC
:104A2000105000F0B3FAD8F81C40AA68031B9A4251
:104A30003ED81444D5E900324FF00009C8F81C40B4
:104A400013605A60C5F80090D8F81030B34201D115
:104A500000F0A8FA89F31188D5E903312846984770
:104A6000302383F311886B69002BD8D000F08EFAC5
:104A70006A69A0EB04094A4582460DD2022000F083
:104A8000DDFA0022D8F81030B34208D1514628464A
:104A9000BDE8F047FFF728BF121A2244F2E712EBF5
:104AA000090938BF4A4629463846FFF7EBFEB5E705
:104AB000D8F81030B34208D01444211AC8F81C00AA
:104AC000A960BDE8F047FFF7F3BEBDE8F08700BF7F
:104AD000A05E0020905E002000207047FEE70000EE
:104AE000704700004FF0FF3070470000BFF34F8F5A
:104AF000024AD368DB03FCD4704700BF003C02408D
:104B000008B5094B1B7873B9FFF7F0FF074B1A691B
:104B1000002ABFBF064A5A6002F188325A601A68FA
:104B200022F480621A6008BD00610020003C02404F
:104B30002301674508B50B4B1B7893B9FFF7D6FFE8
:104B4000094B1A6942F000421A611A6842F4805215
:104B50001A601A6822F480521A601A6842F480625D
:104B60001A6008BD00610020003C02400728F0B533
:104B700016D80C4C0C4923787BB90C4D0E460823F3
:104B80004FF0006255F8047B46F8042B013B13F00C
:104B9000FF033A44F6D10123237051F82000F0BD01
:104BA0000020FCE724610020046100206858000810
:104BB000014B53F8200070476858000808207047E0
:104BC000072810B5044601D9002010BDFFF7CEFF1D
:104BD000064B53F824301844C21A0BB90120F4E7ED
:104BE00012680132F0D1043BF6E700BF68580008B4
:104BF000072810B5044621D8FFF778FFFFF780FF9C
:104C00000F4AF323D360C300DBB243F4007343F0D5
:104C100002031361136943F480331361FFF766FFE6
:104C2000FFF7A4FF074B53F8241000F03DF9FFF7FE
:104C300081FF2046BDE81040FFF7C2BF002010BD35
:104C4000003C024068580008F8B512F00103144611
:104C500042D185182E4A954257D82E4B1B6813F027
:104C6000010352D02C4DFFF74BFFF323EB60FFF70E
:104C70003DFF40F20127032C15D824F001046618EB
:104C8000254C401A40F20117B142236900EB01059F
:104C900024D123F001032361FFF74CFF0120F8BD6D
:104CA000043C0430E7E78307E7D12B6923F4407322
:104CB0002B612B693B432B6151F8046B0660BFF3FA
:104CC0004F8FFFF713FF03689E42E9D02B6923F053
:104CD00001032B61FFF72EFF0020E0E723F4407370
:104CE000236123693B4323610B882B80BFF34F8FE4
:104CF000FFF7FCFE2D8831F8023BADB2AB42C3D0CA
:104D0000236923F001032361E4E71846C7E700BFE6
:104D10000000080800380240003C0240084908B57D
:104D20000B7828B11BB9FFF7EBFE01230B7008BD10
:104D3000002BFCD0BDE808400870FFF7FBBE00BFA9
:104D4000006100204FF480214FF0005000F0AEB819
:104D50000846114600F03ABC012000F037BC0000C4
:104D6000084600F051BC000070B582B0FFF70AFDA4
:104D70000E4E054600F00AF93268904237BF0C4AE1
:104D80000B49516814682EBFD1E9004101315160CF
:104D90000419034641F10001284601913360FFF7F1
:104DA000FBFC0199204602B070BD00BF28610020C5
:104DB0003061002070B582B0FFF7E4FC104E05466C
:104DC00000F0E4F83268904237BF0E4A0D4951684E
:104DD00014682EBFD1E9004101315160041941F13D
:104DE00000010346284601913360FFF7D5FC019985
:104DF0004FF47A7200232046FBF7FAF902B070BD37
:104E0000286100203061002010B50244064BD2B268
:104E1000904200D110BD441C00B253F8200041F86C
:104E2000040BE0B2F4E700BF502800400F4B30B550
:104E30001C6F240407D41C6F44F400741C671C6F9F
:104E400044F400441C670A4C236843F480732360D5
:104E50000244084BD2B2904200D130BD441C00B293
:104E600051F8045B43F82050E0B2F4E70038024008
:104E7000007000405028004007B5012201A9002021
:104E8000FFF7C2FF019803B05DF804FB13B50446B9
:104E9000FFF7F2FFA04205D0012201A900200194F2
:104EA000FFF7C4FF02B010BD70470000704700005C
:104EB00070470000074B45F255521A6002225A60B3
:104EC00040F6FF729A604CF6CC421A60024B012207
:104ED0001A707047003000403C610020034B1B7883
:104EE0001BB1034B4AF6AA221A6070473C610020AE
:104EF00000300040034B1A681AB9034AD2F87428EC
:104F00001A6070473861002000300240024B4FF0B9
:104F10008072C3F8742870470030024008B5FFF76C
:104F2000E9FF024B1868C0F3407008BD38610020EB
:104F300008B5FFF7DFFF024B1868C0F3007008BD2B
:104F40003861002070470000FEE700000A4B0B4864
:104F50000B4A90420BD30B4BDA1C121AC11E22F0E3
:104F600003028B4238BF00220021FCF7F1BD53F849
:104F7000041B40F8041BECE7085A0008C861002035
:104F8000C8610020C861002000F0CAB84FF080431B
:104F9000586A70474FF08043002258631A6102221A
:104FA000DA6070474FF080430022DA6070470000FB
:104FB0004FF0804358637047FEE7000070B51B4B0D
:104FC00001630025044686B0586085620E46FEF7F0
:104FD000E9FF04F11003C4E904334FF0FF33C4E9DF
:104FE0000635C4E90044A560E562FFF7CFFF2B4614
:104FF0000246C4E9082304F134010D4A25658023E3
:105000002046FFF7D9FB0123E0600A4A03750092AE
:1050100072680192B268CDE90223074B6846CDE978
:105020000435FFF7F1FB06B070BD00BFF86000204B
:10503000885800088D580008B94F0008024AD36A02
:105040001843D062704700BF905E00204B684360F9
:105050008B688360CB68C3600B6943614B690362F3
:105060008B6943620B6803607047000008B5234BEF
:1050700023481A6942F0FF021A611A6922F0FF02FE
:105080001A611A691A6B42F0FF021A631A6D42F034
:10509000FF021A651B4A1B6D1146FFF7D7FF02F18D
:1050A0001C0100F58060FFF7D1FF02F1380100F527
:1050B0008060FFF7CBFF02F1540100F58060FFF73D
:1050C000C5FF02F1700100F58060FFF7BFFF02F13C
:1050D0008C0100F58060FFF7B9FF02F1A80100F52F
:1050E0008060FFF7B3FF02F1C40100F58060FFF7B5
:1050F000ADFFBDE8084000F08DB800BF00380240A9
:10510000000002409458000808B500F019FAFFF7B3
:1051100011FBBDE80840FFF7EDBE0000704700003E
:105120000F4B1A6C42F001021A641A6E42F001022F
:105130001A660C4A1B6E936843F0010393604FF0AC
:10514000804331229A624FF0FF32DA6200229A6184
:105150005A63DA605A6001225A611A60704700BFD0
:1051600000380240002004E04FF0804208B5116989
:10517000D3680B40D9B2C9439B07116107D53023CF
:1051800083F31188FFF7FCFA002383F3118808BD2D
:105190001E4B1A6962F0FF021A611A69D2B21A61D3
:1051A0004FF0FF301A695A69586100215A695961F4
:1051B0005A691A6A62F080521A621A6A02F08052C0
:1051C0001A621A6A5A6A58625A6A59625A6A1A6C98
:1051D00042F080521A641A6E42F080521A661A6EB9
:1051E0000B4A106840F480701060186F00F4407033
:1051F000B0F5007F1EBF4FF4803018671967536801
:1052000023F40073536000F073B900BF003802400C
:10521000007000403B4B3C4A1A643C4A4FF440410A
:1052200011601A6842F001021A601A689007FCD5F2
:105230009A6822F003029A60324B9A6812F00C02CC
:10524000FBD1196801F0F90119609A601A6842F4FB
:1052500080321A601A689103FCD55A6F42F001023D
:105260005A67284B5A6F9207FCD5294A5A601A6828
:1052700042F080721A60254A53685804FCD5214BCD
:105280001A689101FCD5234AC3F884201A6842F0B9
:1052900080621A601A681201FCD51F4A9A600322C4
:1052A000C3F88C204FF00062C3F894201B4B1A689F
:1052B0001B4B9A421B4B21D11B4A11681B4A91423E
:1052C0001CD140F203121A60164A136803F00F0350
:1052D000032BFAD10B4B9A6842F002029A609A684B
:1052E00002F00C02082AFAD15A6C42F480425A6445
:1052F0005A6E42F480425A665B6E704740F2037207
:10530000E1E700BF003802400004001000700040D8
:10531000081940021030002400948838002004E06E
:1053200011640020003C024000ED00E041C20F414A
:10533000074A08B5536903F00103536123B1054AD5
:1053400013680BB150689847BDE80840FEF74EBEA1
:10535000003C014040610020074A08B5536903F052
:105360000203536123B1054A93680BB1D068984793
:10537000BDE80840FEF73ABE003C01404061002015
:10538000074A08B5536903F00403536123B1054A82
:1053900013690BB150699847BDE80840FEF726BE77
:1053A000003C014040610020074A08B5536903F002
:1053B0000803536123B1054A93690BB1D06998473B
:1053C000BDE80840FEF712BE003C014040610020ED
:1053D000074A08B5536903F01003536123B1054A26
:1053E000136A0BB1506A9847BDE80840FEF7FEBD4E
:1053F000003C014040610020164B10B55C6904F48C
:1054000078725A61A30604D5134A936A0BB1D06A25
:105410009847600604D5104A136B0BB1506B984740
:10542000210604D50C4A936B0BB1D06B9847E2056B
:1054300004D5094A136C0BB1506C9847A30504D5E9
:10544000054A936C0BB1D06C9847BDE81040FEF74D
:10545000CDBD00BF003C014040610020194B10B59C
:105460005C6904F47C425A61620504D5164A136DE6
:105470000BB1506D9847230504D5134A936D0BB1BA
:10548000D06D9847E00404D50F4A136E0BB1506EEF
:105490009847A10404D50C4A936E0BB1D06E98477F
:1054A000620404D5084A136F0BB1506F9847230468
:1054B00004D5054A936F0BB1D06F9847BDE81040F3
:1054C000FEF794BD003C01404061002008B5034850
:1054D000FEF728FEBDE80840FEF788BD245C0020EA
:1054E00008B5FFF741FEBDE80840FEF77FBD0000AC
:1054F000062108B50846FEF797FE06210720FEF7AD
:1055000093FE06210820FEF78FFE06210920FEF7F4
:105510008BFE06210A20FEF787FE06211720FEF7E4
:1055200083FE06212820FEF77FFE07211C20FEF7C0
:105530007BFEBDE808400C212620FEF775BE00006A
:1055400008B5FFF725FE00F009F8FFF715F8FFF79B
:10555000E5FDBDE80840FFF717BD00000023054A40
:1055600019460133102BC2E9001102F10802F8D1EB
:10557000704700BF406100200B460146184600F00E
:105580002DB8000000F040B8012838BF012010B548
:105590000446204600F030F830B900F007F808B9AA
:1055A00000F00CF88047F4E710BD0000024B1868CB
:1055B000BFF35B8F704700BFC061002008B50620B5
:1055C00000F084F80120FFF789FA0000024B0A4638
:1055D00001461868FFF7BCBB2423002010B5054C1A
:1055E00013462CB10A4601460220AFF3008010BDDD
:1055F0002046FCE700000000024B01461868FFF758
:10560000ABBB00BF24230020024B01461868FFF704
:10561000A7BB00BF2423002010B5013902449042EB
:1056200001D1002005E0037811F8014FA34201D019
:10563000181B10BD0130F2E72DE9F041A3B1C91AE2
:1056400017780144044603F1FF3C8C42204601D9FF
:10565000002009E00578BD4204F10104F5D10CEB0E
:105660000405D618A54201D1BDE8F08115F8018DD9
:1056700016F801EDF045F5D0E7E700001F2938B531
:1056800004460D4604D9162303604FF0FF3038BDA1
:10569000426C12B152F821304BB9204600F030F87C
:1056A0002A4601462046BDE8384000F017B8012BD5
:1056B0000AD0591C03D1162303600120E7E7002418
:1056C00042F82540284698470020E0E7024B014673
:1056D0001868FFF7D3BF00BF2423002038B5074D5B
:1056E00000230446084611462B60FFF7FBF9431CD4
:1056F00002D12B6803B1236038BD00BFC461002014
:10570000FFF7EAB9034611F8012B03F8012B002A31
:10571000F9D170476F72672E6172647570696C6F32
:10572000742E486F6C7962726F475053000000000E
:1057300053544D3332463F3F3F0053544D3332466E
:105740003430780053544D33324634327800535459
:105750004D333246343436585800000001203300AF
:105760000010410001105A000310590007103100C9
:105770000000000030570008130400003A570008EA
:105780001904000044570008210400004E57000887
:1057900040A2E4F1646891060041A3E5F2656992D4
:1057A000070000004261642043414E496661636521
:1057B00020696E6465782E00000100000001FF0082
:1057C000006400400068004080000000008000008D
:1057D0000000800000000000000000001D24000800
:1057E000A92C0008B52B00082D240008612400080E
:1057F0005D260008312400084124000835240008F3
:105800003D240008392400088525000845240008A7
:10581000A92F00085524000859250008009600000B
:105820000000000000000000000000000000000078
:1058300000000000394500082545000861450008C2
:105840004D45000859450008454500083145000808
:105850001D4500086D4500086330000058580008D9
:10586000E85E0020F86000200040000000400000DA
:1058700000400000004000000000010000000200A5
:1058800000000200000002006D61696E0069646C36
:1058900065000000A001812A00000000AAA9AAAAB0
:1058A00050000124EFFF0000007700000090090085
:1058B0001000004A000000009AAAAAAA00000000F6
:1058C000FBFF000000000000000099000000000045
:1058D00000000000AAAAAAAA00000000FFFF000022
:1058E00000000000000000000000000000000000B8
:1058F000AAAAAAAA00000000FFFF00000000000002
:10590000000000000000000000000000AAAAAAAAEF
:1059100000000000FFFF0000000000000000000089
:105920000000000000000000AAAAAAAA00000000CF
:10593000FFFF000000000000000000000000000069
:1059400000000000AAAAAAAA00000000FFFF0000B1
:105950000000000000000000000000000000000047
:105960000A0000000000000003000000000000002A
:1059700000000000ACA8FF7F010000000000000054
:105980000B04000000000000000007000000000001
:1059900040420F00FE2A0100D2040000FF00000078
:1059A000245C0020282300200000000000000000EC
:1059B00000000000000000000000000000000000E7
:1059C00000000000000000000000000000000000D7
:1059D00000000000000000000000000000000000C7
:1059E00000000000000000000000000000000000B7
:1059F00000000000000000000000000000000000A7
:085A000000000000000000009E
:00000001FF
